:100000000C9426040C9443040C9443040C94430471
:100010000C9443040C9443040C9443040C94430444
:100020000C9443040C9443040C9443040C94430434
:100030000C9443040C9443040C9443040C94430424
:100040000C94F2070C9461050C9443040C94430443
:100050000C9443040C9443040C9443040C94430404
:100060000C9443040C9443040C9443040C944304F4
:100070000C9443040C9443040C9443040C944304E4
:100080000C9443040C9443040C944304E11DB91FE5
:10009000E61DA41FFD1DFD1D371E3F1E711EC01E47
:1000A0003C1EB91FB91F551F671F851F931FB91F1E
:1000B000B91FB91FB91FB91FB91FB91FB91FB91F80
:1000C000B91FB91FB91FA81FAA1FAF1F45617379B8
:1000D000436F6E74726F6C00204C4300696E636FE7
:1000E0006D70617469626C6520485700312E342E42
:1000F00030000102031304050611070809120A0063
:100100000B0C100F0E0D010101050D1F0C04040E48
:100110001F04041F0E040006091717090600000635
:1001200009121412090603070F1E1C1810000305FC
:100130000912141810000707070707070707070524
:100140000505050505071C101817150705071C10E0
:100150001817110202021C101812140605021C10B6
:100160001817140601061C101815150701011C109C
:100170001816110201061C101816110204071C1093
:10018000181216020207040A110A0A0E00000C17C0
:10019000141714170C001C101810160505051F0A5B
:1001A0000A0A0A0A1F000E11111F1B1B1F0002065C
:1001B0000F1F0F060200080C1E1F1E0C08000E0E5B
:1001C0000E0E1F0E0400040E1F0E0E0E0E00202039
:1001D000202020200000204D4D4920200000204DEF
:1001E0004D012020000020444343202000002053E4
:1001F000544F5020000053484F52542100002048D3
:10020000414C54200000000000000000000020507D
:10021000524F4720000052455345542000007E0EA7
:100220000E0E0E1B1B1C0E1B1B7E0E0E0E0E232D08
:10023000004144523A20256C6420202020202020B8
:10024000202020002D2D2D2D202000252D3564006F
:1002500025336400202001022020202020202000BF
:10026000252D356400252D31312E31317300414269
:10027000434445464748494A4B4C4D4E4F505152D6
:10028000535455565758595A30313233343536371E
:1002900038392E2C3A2D2B232F3D3C7C3E20004D0F
:1002A0004D20492020313420004D4D20492020325E
:1002B0003761004D4D20492020323762004D4D20DE
:1002C000012020313420004D4D20012020323761A3
:1002D000004D4D200120203237620044434320204E
:1002E0002031342000444343202020323820004471
:1002F0004343202031323820004C6F636D656E75AA
:1003000000000000000000000044434320686F6FBD
:10031000666473706F6F7200004C434420766572A0
:100320006C69636874696E67004C6F6B436F6E74C1
:10033000726F6C00000000000045786974000000D6
:100340000000000000000000004B69657A656E2027
:1003500000000000000000000044617461666F72DC
:100360006D61740000000000004E61616D2020206E
:10037000202020000000000000496E766F6572208A
:100380002020200000000000004D656E75204C6F9D
:10039000636F0000000000000050726F6772616DB3
:1003A0006D6174696F6E0000004C756D696E6F73DE
:1003B0006974650000000000004C6F6B436F6E7441
:1003C000726F6C0000000000004578697400000046
:1003D00000000000000000000053656C6563746954
:1003E0006F6E20000000000000466F726D61742087
:1003F000646F6E6E65657300004E6F6D2020202067
:10040000202020000000000000536169736965200E
:100410002020200000000000004C6F6B204D656E16
:10042000FC000000000000000044434320486175C8
:100430007074676C65697300004C43442042656CBE
:100440006575636874756E67004C6F6B436F6E748F
:10045000726F6C00000000000045786974000000B5
:1004600000000000000000000041757377E4686C34
:10047000656E20000000000000446174656E666FC8
:10048000726D617400000000004E616D65202020D7
:1004900020202000000000000045696E7472616732
:1004A000202020000000000000547261696E206D61
:1004B000656E75000000000000444343204D6169F3
:1004C0006E20547261636B00004C4344206C69677A
:1004D0006874696E67000000004C6F6B436F6E7448
:1004E000726F6C0000000000004578697400000025
:1004F00000000000000000000073656C656374205C
:100500000000000000000000004461746120666F7C
:10051000726D617400000000004E616D6520202046
:10052000202020000000000000456E747279202019
:10053000202020000000000000202D2D2D2D002562
:10054000357500536F6674772E205600312E342E89
:1005500030005365724E722E2025386C75003A209B
:100560000025357500253364002534643A20002DBC
:100570002D2D0025336400204F4B2020202000200B
:1005800020202020202000696E636F6D7061742E22
:1005900020466F726D617400496E636F6D702E201E
:1005A000466F726D6174202000466F726D61742019
:1005B000696E636F6D7061742E00696E6B6F6D7024
:1005C00061742E20466F726D6174002E2E2E20777E
:1005D000616974696E67202E2E2E2000233D6465AC
:1005E0006C657465000000000000000000286E6F5C
:1005F00020656E74727929000000000000002E2E24
:100600002E2064656C6574696E67202E2E2E002086
:100610006661756C740000000000000000000000BE
:1006200020444343206F6E6C7921000000000000DD
:10063000002A3D446973636F6E742E200000000031
:1006400000002070726F6772616D696E6700000054
:100650000000002D73686F7274206369726375699E
:10066000742D20002E2E2E207761636874656E2015
:100670002E2E2E2020233D77697373656E000000B7
:10068000000000000000286765656E20696E766FC7
:1006900065722900000000202E2E2E2077697373CA
:1006A000656E202E2E2E000020666F7574000000EF
:1006B00000000000000000000020416C6C65656EC9
:1006C000204443432100000000002A3D204166628F
:1006D00072656B656E0000000000002050726F674D
:1006E00072616D6D6572656E000000002D2D4B6F9F
:1006F0007274736C756974696E672D2D0050617426
:1007000069656E74657A0000000000000000233DFA
:100710007375707072696D6572000000000000767C
:100720006964650000000000000000000000000097
:100730005375707072657373696F6E00000000000E
:100740000020457272657572000000000000000014
:1007500000002044434320756E697175656D656EB8
:100760007400002A3D4162616E646F6E20200000BB
:10077000000000002050726F6772616D6D617469D6
:100780006F6E0000002D436F7572742D6369726384
:100790007569742D20002E2E2E2077617274656E7F
:1007A000202E2E2E202000233D4CF6736368656EAC
:1007B0000000000000000000286B65696E2045699C
:1007C0006E7472616729000000202E2E2E206CF6B8
:1007D00073636865202E2E2E2000204665686C65A8
:1007E0007200000000000000000000206E75722002
:1007F00066FC722044434321000000002A203D2073
:10080000416262727563680000000000002050724F
:100810006F6772616D6D696572756E6700002D2D71
:10082000204B75727A7363686C75DF202D2D005B29
:100830006E6F206D6573736167655D005B756E6BD0
:100840006E6F776E206572726F725D0011241FBE2D
:10085000CFEFD0E1DEBFCDBF11E0A0E0B1E0E0E33B
:10086000FBE400E00BBF02C007900D92A832B10775
:10087000D9F713E0A8E2B1E001C01D92A034B1079E
:10088000E1F70C947D040C94000081E08093290131
:100890000895482F90912801981731F0963021F053
:1008A000953029F4863019F080E090E00895409367
:1008B0002801453021F460E280E00E94FC1F409155
:1008C0002801463021F460E280E00E94FC1F0E9473
:1008D000450481E090E008950895809128019927CA
:1008E00008950E94AB1D0E94D90F80912901882391
:1008F00011F40E94440BA8950895CFEFD0E1DEBF1C
:10090000CDBF0E94281B0E941D050E9442057894BD
:100910000E94A2070E944E1BFC0184810E94AD0B25
:100920006CEC70E082E00E94D00B0E94641B82306D
:1009300079F00E94641B813059F060E081E00E94F0
:100940005A0A6CED70E082E00E94D00BA895FECFB1
:1009500068ED70E082E00E94D00B60E081E00E94D0
:100960005A0A66E582E00E94B20B6CEE70E082E00B
:100970000E94D00B0E944E1B8C0181E00E945909FD
:10098000882319F081E00E94511B82E00E945909DE
:10099000882319F080E00E94511B83E00E945909CE
:1009A000882319F082E00E94511B84E00E945909BB
:1009B000882329F083E00E94511B01C0A8950E9462
:1009C000CA1C8823D9F3F80181859285892BC9F047
:1009D0000E94640CEC0144969E01215F3F4FAC01E4
:1009E000B901F801818592850E940221BC01892B01
:1009F00029F0F801818592858A8B9B8B61157105A1
:100A000019F4F801628173818FEF0E94C51B81E0A8
:100A100011C00E94F40F0E940A0AFFEF8F3F9F0748
:100A2000C1F70E947104809129018823A1F31092DB
:100A3000290180E00E94DE0DEECF8FE78ABB1BBA52
:100A400080E187BB18BA80EF84BB8FEF85BB8BEB4F
:100A500081BB8CEC82BB86E082B987EF83B980933F
:100A6000610081EF809362008FE18093640089E1EF
:100A7000809365000E94D308A89588E181BD8CE031
:100A800081BD08950E94561B9B01AC0193E0E92FA4
:100A9000FF27EC5CFE4F822F8F77808387E056958F
:100AA0004795379527958A95D1F7915097FFEFCFC6
:100AB00087B3807F87BB88B3807F88BB84EE8DB986
:100AC00008951F920F920FB60F9211242F933F9308
:100AD0004F935F936F937F938F939F93EF93FF93C6
:100AE00080910001909101018F5F9F4F71F0BB9A3F
:100AF000809100018FB9769B0BC0BB9810922A01A0
:100B0000109231011092300103C0BB988FEF8FB962
:100B10007FB177FF7FC08091320190913301892BA3
:100B2000E1F080912E018F5F80932E0180912E0144
:100B3000803210F010922E0190912E0180912F01A1
:100B4000981759F480912F018F5F80932F01809126
:100B50002F01803210F010922F018091300190917E
:100B60003101855D924061F058F080912D018F5FD9
:100B700080932D0180912D01843010F010922D0171
:100B80001092330110923201109231011092300113
:100B900060912601761721F481E080932A0171C0CB
:100BA00010922A01472F55279A012F773070862FF0
:100BB00099272817390721F07F3F11F06F3F61F423
:100BC00090912E0189E0989FC00111248B549E4F73
:100BD00090933301809332014F775070862F99277D
:100BE0004817590709F04DC090912C0180912D01B3
:100BF000981749F090912D0189E0989FC001112428
:100C00008B529D4F02C08CEA91E09093310180930A
:100C1000300137C020912A01822F99278130910518
:100C200031F0813091056CF106975CF516C02F5FAD
:100C300020932A01703419F410922B0122C07134D0
:100C400011F481E007C0723411F482E003C0733400
:100C500091F483E080932B0114C0E22FFF27809151
:100C60002B01992702968E179F0744F0EE5CFE4FEA
:100C70008081781719F010922A0103C02F5F20930A
:100C80002A0180912A01882339F4809130019091C2
:100C90003101892B79F003C0872F99270DC0E0918E
:100CA0003001F091310181919927F0933101E09366
:100CB000300102C08FEF9FEF9093010180930001FC
:100CC0008091320190913301855D924020F0109225
:100CD000330110923201E0913201F09133013097EB
:100CE00029F07193F0933301E0933201FF91EF917A
:100CF0009F918F917F916F915F914F913F912F9134
:100D00000F900FBE0F901F901895DC0180912C0161
:100D1000282F332780912D0199270197281739070C
:100D200041F080912C01833039F480912D0188238A
:100D300019F480E090E0089590912C0189E0989F4B
:100D4000F0011124EB52FD4F98E08D918193915069
:100D500097FFFBCF80912C018F5F80932C018091B6
:100D60002C01843010F010922C0181E090E0089565
:100D70000895FC01ACEAB1E098E081918D93915027
:100D800097FFFBCF08959C0190912E0180912F0138
:100D9000981719F480E090E00895D90121153105E4
:100DA00011F4C9010895F89490912F0189E0989F5A
:100DB000F0011124EB54FE4F98E081918D939150F6
:100DC00097FFFBCF80912F018F5F80932F01809140
:100DD0002F01803210F010922F017894C9010895EC
:100DE000089500000000000000000895882341F0ED
:100DF000809165008460809365000E94F1060895EB
:100E0000809165008B7F80936500089508959B0114
:100E1000AC018091FB029091FC02A091FD02B09187
:100E2000FE0282179307A407B507A0F08091FB028A
:100E30009091FC02A091FD02B091FE02821B930BE7
:100E4000A40BB50B80509041A040B040A0F080E0D2
:100E500090E008958091FB029091FC02A091FD0228
:100E6000B091FE02281B390B4A0B5B0B2050304F10
:100E70004F4F5F4F18F081E090E0089580E090E0E0
:100E800008950895EF92FF920F931F93AA27BB270F
:100E9000E090FB02F090FC020091FD021091FE0236
:100EA000E80EF91E0A1F1B1F01C0A895C801B70153
:100EB0000E9407078823C9F31F910F91FF90EF90BD
:100EC00008950F931F93CF93C82F162F042F80914F
:100ED00065008D7F8093650080E00E94F6068AB3EE
:100EE0008F608ABB8BB3807F9C2F92959F70892BDC
:100EF0008BBB112321F080916500816003C080913C
:100F000065008E7F8093650081E00E94F60680E098
:100F10000E94F606002329F088E090E00E94420734
:100F20000DC08BB3807FCF708C2B8BBB0E94F106E2
:100F300081E00E94F606802F0E94F606CF911F9155
:100F40000F91089588E290E00E94420741E060E03E
:100F500080E30E94610741E060E080E30E94610756
:100F600041E060E080E30E94610741E060E080E2F0
:100F70000E94610788E20E94500A88E00E94500A9D
:100F800081E00E94500A86E00E94500A8CE00E9494
:100F9000500A66EC71E080E00E94890B6EE971E016
:100FA00081E00E94890B66EA71E082E00E94890B71
:100FB0006EE871E083E00E94890B6EE771E084E0E7
:100FC0000E94890B66E771E085E00E94890B6EE65E
:100FD00071E086E00E94890B66E671E087E00E947E
:100FE000890B08951F920F920FB60F9211241F9331
:100FF0002F933F934F935F936F937F938F939F9321
:10100000AF93BF93EF93FF9380913A01882309F048
:10101000B8C081E080933A017894809138018F5F65
:1010200080933801282F237009F0A9C086958695F2
:101030008770992783309105C1F1843091052CF494
:10104000009759F00197E9F09AC08530910509F4AD
:1010500060C0079709F491C092C08091FB02909103
:10106000FC02A091FD02B091FE020196A11DB11DEE
:101070008093FB029093FC02A093FD02B093FE02CA
:101080007EC08091FB029091FC02A091FD02B09184
:10109000FE0281709070A070B070892B19F00E94D0
:1010A0006C096DC00E942D096AC0809139018823A6
:1010B00009F465C08AB3807F8ABB822F0E94F6063E
:1010C00080916500826080936500809165008E7FCD
:1010D000809365000000000081E00E94F60619B3CD
:1010E00080E00E94F6061295107F0E94F10681E0D2
:1010F0000E94F60689B38F70182B80E00E94F606D6
:10110000812F992787FD90958827990F881F992708
:1011100031C060913901662391F59091FF02809171
:101120000003981789F010910003E12FFF27E15089
:10113000FD4F82811F5F103108F0162F803891F427
:101140008091FF02811719F480E090E013C0E12F35
:10115000FF27E150FD4F82811F5F103108F0162FED
:10116000462F02C0462F61E00E94610710930003E2
:1011700081E090E08093390102C00E94F009109252
:101180003A01FF91EF91BF91AF919F918F917F9124
:101190006F915F914F913F912F911F910F900FBED3
:1011A0000F901F90189510927D0017BE11BE89E612
:1011B00083BF87B7816087BF0895EF92FF920F9337
:1011C0001F93AA27BB27E090FB02F090FC0200913E
:1011D000FD021091FE02E80EF91E0A1F1B1F02C03D
:1011E0000E947104C801B7010E9407078823C1F358
:1011F0001F910F91FF90EF900895282F220F6111FA
:101200002160822F83708150823028F424FF02C035
:101210002E6001C0217F822F9927089590913D0172
:10122000E92FFF27E35CFE4F8283892F8F5F809336
:101230003D01883010F010923D0190913E01809167
:101240003D01981741F4892F8F5F80933E018830CC
:1012500010F010923E01089508950F931F9311B15D
:10126000812F8074682F80913B010E94FD08082F18
:1012700080933B011078612F80913C010E94FD0812
:1012800080933C01007C807C003829F4882339F06D
:10129000803C61F408C0003449F4803C11F484E1DE
:1012A00003C0882319F485E10E940E091F910F9154
:1012B0000895843118F080E090E0089520E030E057
:1012C000E82FFF27E95BFE4F8081882311F021E0A2
:1012D00030E0C90108950895FF920F931F93CF93B3
:1012E00080916001E82FFF27E55AFE4F008113B37C
:1012F0001083FF2480916001E82FFF27EE0FFF1F6E
:10130000EE0FFF1FEF0DF11DEE50FF4FC49110FDCA
:1013100031C000FF14C0C23129F481E10E94590993
:10132000882331F48C2F0E940E09C43108F043C089
:10133000EC2FFF27E95BFE4F81E080833CC0C43186
:10134000D0F5EC2FFF27DF01A95BBE4F9C919F5F7B
:101350009C93992311F49F5F9C937197329758F552
:1013600080915801893738F180915901893718F1F6
:1013700085E01FC0C43128F4EC2FFF27E95BFE4F46
:10138000108200FD18C08C2F80680E940E090E94F8
:101390006D04853081F4C13121F482E10E94590944
:1013A00005C0C23141F481E10E945909882319F432
:1013B00086E00E94490416950695F39483E08F1504
:1013C00008F098CF809160018F5F80936001853035
:1013D00010F010926001CF911F910F91FF9008952E
:1013E00090916001943029F485B3806F85BB979804
:1013F0000895979A85B38F7020E130E002C0220FE4
:10140000331F9A95E2F7922F9095907F892B85BB99
:101410000895089580913D0120913E01821719F4AD
:101420008FEF9FEF0895E22FFF27E35CFE4F82814D
:10143000482F5527822F8F5F80933E01883010F010
:1014400010923E01CA0108950895482F05C0809169
:101450000003882381F4A8958091FF02282F332769
:10146000809100039927019728173907A1F38091EC
:10147000FF028F3061F3F8948091FF02E82FFF277D
:10148000E150FD4F42838091FF028F5F8093FF0206
:101490008091FF02803110F01092FF02789408953D
:1014A0001F93182F80E80E94250A812F0E94250A89
:1014B0001F9108958295880F880F807C860F806821
:1014C0000E94500A08950E945A0A8EE00E94500A13
:1014D00008958CE00E94500A0895FF920F931F9385
:1014E000CF93F82E60912203809121030E945A0A23
:1014F000C0E001E113E080912303C81778F4FF20D6
:1015000021F0F80161918F0101C060E282E00E9448
:10151000B20BCF5F80912303C81788F3CF911F913F
:101520000F91FF90089590932C0380932B03892BA8
:1015300089F170932A0360932903CB01AA27BB2763
:101540002091FB023091FC024091FD025091FE027D
:10155000280F391F4A1F5B1F209325033093260352
:101560004093270350932803809124038E7F809318
:101570002403211531054105510561F42F5F3F4FCB
:101580004F4F5F4F2093250330932603409327034B
:101590005093280308950895AF92BF92CF92DF929F
:1015A000EF92FF920F931F93CF93DF93D82EC62E07
:1015B000EA0181E1E82E83E0F82E10922C031092CC
:1015C0002B0381E08D1568F1EFE0E61750F141152E
:1015D000510539F1FA0101900020E9F731970E2FFA
:1015E000041B013108F000E16C2D8D2D0E945A0A78
:1015F0005701002361F0102F8881F50181935F016D
:101600008991682F82E00E94B20B1150A9F7F7016F
:10161000D08AC18A028B64EF71E08DE69AE00E9465
:10162000930ADF91CF911F910F91FF90EF90DF9080
:10163000CF90BF90AF900895CF93DF93CDB7DEB733
:10164000A0970FB6F894DEBF0FBECDBF282FDE01E6
:10165000119690E0FA014F5F5F4F8491882321F04B
:101660008D939F5F9F31B0F31C92AE014F5F5F4F30
:10167000822F0E94CC0AA0960FB6F894DEBF0FBE50
:10168000CDBFDF91CF91089580912B0390912C03D2
:10169000892BA9F16091250370912603809127037E
:1016A000909128030E940707882349F18091240321
:1016B000E0912B03F0912C03817009958091240314
:1016C00091E08927809324038091290390912A0334
:1016D0009C01442755278091FB029091FC02A09128
:1016E000FD02B091FE02820F931FA41FB51F8093CD
:1016F000250390932603A0932703B093280308950E
:10170000089510922C0310922B0381E00E94500A3E
:1017100008950F931F93CF93DF93EB018830C0F4AC
:10172000992723E0880F991F2A95E1F780640E948A
:10173000500A07E010E0FE01219684910E94250ADC
:101740000150104017FFF7CF60E0862F0E945A0A21
:10175000DF91CF911F910F910895813308F080E3BD
:1017600081BF08958230D1F467FF15C0643E31F027
:10177000663F41F06C3F51F0643C11F461EE0BC0E8
:10178000663D11F46FEE07C06C3D11F465EF03C0C8
:101790006F3D09F462EE862F0E94250A0895089590
:1017A0001F93CF93DF93182FEB01FB016491662306
:1017B00049F0812F0E94B20B2196FE018491682F7F
:1017C0008823B9F7DF91CF911F9108951F93CF938D
:1017D000DF93182FEB018881882341F08991682FCE
:1017E000812F0E94B20B88818823C1F7DF91CF91AE
:1017F0001F9108951F93CF93DF93CDB7DEB7C055E8
:10180000D0400FB6F894DEBF0FBECDBF67961FADB8
:10181000679769968EAD9FAD6997AE01475A5F4F46
:10182000BC01CE0101960E942522BE016F5F7F4F51
:10183000812F0E94E60BC05BDF4F0FB6F894DEBF2E
:101840000FBECDBFDF91CF911F9108951F93CF930E
:10185000DF93CDB7DEB7C055D0400FB6F894DEBFEA
:101860000FBECDBF67961FAD679769968EAD9FADD2
:101870006997AE01475A5F4FBC01CE0101960E94A5
:101880004E22BE016F5F7F4F812F0E94E60BC05B2F
:10189000DF4F0FB6F894DEBF0FBECDBFDF91CF9103
:1018A0001F910895823019F40E940A0A08958FEF5B
:1018B0009FEF08950895E82FFF27EF70F070E25E24
:1018C000FD4F84919927089581E691E008958091D4
:1018D0006F0182FF05C080916301909164010895BA
:1018E00080916101909162010895089580916F0146
:1018F000826080936F0108950F931F93CF93DF93BE
:10190000C1E6D1E080916F0199278C0101701070C0
:1019100080FF03C080E090E021C06091670170917A
:1019200068018091690190916A01611571058105D5
:10193000910531F00E940707882311F4C8010EC0F9
:101940001A821B821A8A1B8A10926201109261010C
:101950001E861C8A0E94450481E090E0DF91CF91B1
:101960001F910F9108959C018091630190916401F2
:10197000892B11F4C90108952F703F7B77FD3064E6
:10198000CB018F70907044E0880F991F4A95E1F762
:10199000822B932B08950895FC0180916101909111
:1019A00062012091630130916401E817F907F9F4AD
:1019B00060937101232BB1F08091650190916601D4
:1019C000F4E096958795FA95E1F7BC016F70707019
:1019D000892F99278695869580FD7068CA010E9497
:1019E000B30C0FC050936601409365010EC0E2171F
:1019F000F30759F4BA0180916501909166010E9444
:101A0000B30C90936601809365010E94450408958C
:101A10009C01892B69F410926F011092670110925A
:101A200068011092690110926A010E947C0C08956D
:101A30006093710150936601409365018091FB02B0
:101A40009091FC02A091FD02B091FE0288519C4F42
:101A5000AF4FBF4F81608093670190936801A0935F
:101A60006901B0936A0180916F0182FF09C08160B2
:101A70008B7F80936F01309364012093630107C0D3
:101A80008E7F80936F0130936201209361010E94E9
:101A900045040895089520916F012B7F21602093C4
:101AA0006F0190936401809363018091650190912F
:101AB00066010E94B30C90936601809365010E94B9
:101AC00045040895809370010E945B0C809372011D
:101AD0000E9445040895CF93C82F882319F06EE51E
:101AE00071E002C06EE771E084E00E94890BCC23B4
:101AF00019F066E571E002C066E771E085E00E94DA
:101B0000890BCC2319F06EE471E002C06EE671E03F
:101B100086E00E94890BCC2319F066E471E002C0D4
:101B200066E671E087E00E94890BCF910895CF931C
:101B3000DF93C82FDD27C4FF02C083E001C085EA20
:101B40000E94250AC0FF02C084E001C085EA0E940D
:101B5000250AC1FF02C085E001C085EA0E94250A6E
:101B6000C2FF02C086E001C085EA0E94250AC3FFC9
:101B700002C087E001C085EA0E94250ADF91CF916B
:101B80000895809381010E9445040895882319F0E7
:101B900066E271E002C06EE271E082E00E94890BB1
:101BA00008950895882319F066E371E002C06EE39A
:101BB00071E081E00E94890B089508950F931F93AF
:101BC000CF9301E611E0C0918101CC2399F060E050
:101BD00081E00E945A0A8C2F81500E94D01ABC01C9
:101BE00082E00E94D00B1092810188EE93E00E9467
:101BF000DD0802C0882319F00E94810B03C0682F02
:101C00000E945A0A8091610190916201892BF9F03A
:101C10000E944E1BFC018281938140916101509191
:101C200062018417950749F42185328580917301FB
:101C3000909174012817390751F0428353838091A2
:101C4000730190917401818792870E94F31A209109
:101C50006101309162012115310529F4F8012483D5
:101C60003583108A178680916F0182FD0DC08091A7
:101C70006B0190916C01A0916D01B0916E01009784
:101C8000A105B10519F105C06EE272E082E00E9483
:101C9000D00B80916B0190916C01A0916D01B0917E
:101CA0006E01BF93AF939F938F9381E392E09F93D5
:101CB0008F9382E08F930E94260C8DB79EB7079674
:101CC0000FB6F8949EBF0FBE8DBF43C021153105DE
:101CD00031F464E472E082E00E94D00B18C03F93BC
:101CE0002F938BE492E09F938F93C2E0CF930E9457
:101CF000260C80916F010F900F900F900F900F9016
:101D000080FF02C08C2F01C080E20E94250AC09192
:101D100070010E946D04853010F085E00EC08330A4
:101D200061F48C2F99278370907023E0880F991F9E
:101D30002A95E1F782539E4F08C0992703E0880F48
:101D4000991F0A95E1F782519E4FBC0182E00E94E3
:101D5000D00B6CE080E00E945A0A809171019927B3
:101D60008F7790709F938F9380E592E09F938F93EE
:101D700082E08F930E94260C8091700199278370D6
:101D800090700F900F900F900F900F90019781F42B
:101D900083E10E945909882339F06EE071E080E008
:101DA0000E94890B80E001C080E20E94250A0FC0DA
:101DB00080E00E94250A8091710187FF03C066ECD4
:101DC00071E002C06EEB71E080E00E94890B0E941E
:101DD0006D04C82F813049F488E00E949B1AAC0141
:101DE00060E08C2F0E941C0BE0C040E050E060E0FF
:101DF000862F0E94CC0AC0E08AE00E9459098823FD
:101E000071F08091630190916401892B39F4809184
:101E10007001992783709070039709F4C1E060E026
:101E200081E00E945A0A80916B0190916C01A0910F
:101E30006D01B0916E010097A105B10509F442C092
:101E40008DE00E945909882329F48EE00E945909E7
:101E5000882381F184E592E09F938F93C2E0CF9332
:101E60000E94260C8DE00E9459090F900F900F9050
:101E7000882379F066E371E081E00E94890B6EE2CD
:101E800071E08C2F0E94890B6CE271E082ED9DE085
:101E90000EC06EE371E081E00E94890B66E271E0A2
:101EA0008C2F0E94890B6CE271E086EC9DE00E9411
:101EB000930A7BC086E00E949B1ABC0182E00E94CC
:101EC000D00B44C08091630190916401009769F147
:101ED0009F938F9380E692E09F938F9382E08F93FE
:101EE0000E94260C809165019091660114E0969500
:101EF00087951A95E1F7282F2F70892F99278695B6
:101F000086950F900F900F900F900F9080FD20619D
:101F1000822F0E94970DCC2321F08CE30E94250A8A
:101F200015C080E20E94250A2CC085E791E09F93AE
:101F30008F9385E692E09F938F9382E08F930E9428
:101F4000260C0F900F900F900F900F90CC23C9F09C
:101F50008091630190916401892B99F480916501CE
:101F600090916601A4E096958795AA95E1F78F7008
:101F700080610E94970D81E00E946B0D66E871E020
:101F800011C0209165012F708091650190916601CB
:101F900097FD2061822F0E94970D80E00E946B0DBB
:101FA0006EE871E083E00E94890BCF911F910F9141
:101FB0000895609167017091680180916901909125
:101FC0006A01611571058105910561F00E9407079D
:101FD000882341F010926701109268011092690104
:101FE00010926A0108950895AF92BF92CF92DF9246
:101FF000EF92FF920F931F93CF93DF93CDB7DEB78E
:102000002C970FB6F894DEBF0FBECDBF8C0121E632
:10201000C22E21E0D22E86E0FE01319611928A95E1
:10202000E9F701311105DCF40F3011050CF0EFC0B8
:102030000A30110509F415C20B3011053CF40115E5
:10204000110509F410C117FD1BC220C10C30110588
:1020500009F460C00D3011050CF07BC048C105319A
:102060001105C1F1063111057CF40231110509F4A5
:10207000EAC0023111050CF4E8C003311105B9F1D1
:102080000431110591F0FCC10F3811054CF40D38E5
:1020900011050CF05EC00A38110509F4EFC1F0C15A
:1020A0000339110509F4EAC1EBC180917101992747
:1020B0008F779070209172013327821793070CF06D
:1020C000DFC10E946D04833009F0DAC18091710193
:1020D0008F5F1DC020917101822F99278F7790709B
:1020E000892B09F4CDC1215020937101C7C1809182
:1020F0007001992783709070019729F46EE071E068
:1021000080E00E94890B8091710180958078809396
:102110007101B4C18AE00E945909882399F0809125
:10212000630190916401892B69F080916501909120
:10213000660120E030E48227932790936601809324
:1021400065019CC1809165019091660120E030E8B5
:1021500074C086E097E0A92EB12CAC0EBD1EF5012F
:1021600011928A95E9F780916B0190916C01A09191
:102170006D01B0916E010097A105B10509F445C04C
:10218000E0906B01F0906C010894E108F108EE0C0E
:10219000FF1CC8018F7790700E9721F481E090E0CA
:1021A000E82AF92A07FF16C01A8660E070E0CB0122
:1021B0000E94930A6EE971E081E00E94890B66EA51
:1021C00071E082E00E94890BF60112861386148664
:1021D000158602C081E08A878E2D8F778F83EE0C63
:1021E000EF2CEE1CFF08F1948E2D8F778887EE0C74
:1021F000EF2CEE1CFF08F1948E2D83708987A501CA
:1022000066E080E00E94951D39C107FD37C1A3EF4C
:10221000FA2EF00E8AE00E945909882319F0F7EF90
:10222000FF2EF00E21E030E002C0220F331FFA949F
:10223000E2F7809165019091660182279327F6016C
:10224000848395831BC143E006C08AE00E9459093C
:10225000882321F042E060E280E002C0482F60E283
:102260000E94FC1F0BC180916B0190916C01A091A9
:102270006D01B0916E010097A105B10539F48FEFA2
:102280000E94691A81E00E94DE0DFAC080916B0104
:1022900090916C01A0916D01B0916E019C01AD0116
:1022A000E3E0220F331F441F551FEA95D1F7280F93
:1022B000391F4A1F5B1F280F391F4A1F5B1FC801A8
:1022C000AA2797FDA095BA2F280F391F4A1F5B1F19
:1022D0002030F8E23F07F0E04F07F0E05F070CF036
:1022E000CFC0F6012287338744875587C7C071E680
:1022F000E72E71E0F72E86E0AE01495F5F4FFA01ED
:1023000011928A95E9F700916B0110916C0120916F
:102310006D0130916E01609163017091640101154E
:1023200011052105310509F48FC06115710581F191
:10233000A0906101B0906201C501AA27BB27801758
:102340009107A207B30741F0CB01AA27BB2780174B
:102350009107A207B307E1F480916F018E7FF60128
:102360008687809161018F778F83AA0CAB2CAA1C82
:10237000BB08B1948A2D8F77888765E080E00E9442
:10238000951DF60112821382109262011092610172
:1023900080916101909162019C01442755278091B1
:1023A0006B0190916C01A0916D01B0916E016091F3
:1023B0006F01281739074A075B0731F481E0682766
:1023C0006B7FF701668748C06C7FF7016687128ACA
:1023D000138A148A6091750181E00E945A0A80E094
:1023E0000E949B1ABC0182E00E94D00B80916F0179
:1023F000992796958795969587959C0121703070C1
:1024000080FD12C0F7012283338324833583309308
:10241000620120936101178660916B0170916C01DC
:102420008FEF0E94C51B0BC040916B0150916C0156
:1024300060916101709162018FEF0E94F41B8091A5
:102440006F018B7FF70106C0672B29F480916F0124
:102450008460F6018687F701128613861486158636
:102460000DC010926B0110926C0110926D011092D0
:102470006E0180916F018B7F80936F010E944504F4
:102480002C960FB6F894DEBF0FBECDBFDF91CF9173
:102490001F910F91FF90EF90DF90CF90BF90AF9082
:1024A0000895FB0121E057FF04C020E050954195BD
:1024B0005F4F8330910549F18430910534F48130C8
:1024C000910591F0029729F12AC08430910519F005
:1024D000059761F024C081818F5F818399278417DC
:1024E0009507ECF0222359F0118219C081818150A7
:1024F000818399278417950794F0222321F0842F54
:10250000815081830CC021830AC012821382168AF3
:1025100006C090E08281882309F491E0928380E0F4
:1025200090E008950F931F93CF93DF938C010E9447
:10253000670CEC01009731F469E375E082E00E94DA
:10254000D00B0FC09F938F938FE395E09F938F9352
:1025500082E08F930E94260C0F900F900F900F90A7
:102560000F900115110521F0B80182E00E94D00BF7
:10257000CE01DF91CF911F910F9108950F931F937B
:10258000CF93DF93EC018B01009731F097FD35C0BD
:102590000297029790F52BC060E081E00E945A0AF2
:1025A000F8018281882359F463E475E082E00E9497
:1025B000D00B6CE475E082E00E94D00B18C00E9442
:1025C000561BDC01CB01BF93AF939F938F9382E5A2
:1025D00095E09F938F9382E08F930E94260C8DB796
:1025E0009EB707960FB6F8949EBF0FBE8DBF40E012
:1025F00050E0B801CE010E94511280E090E0DF91DE
:10260000CF911F910F9108958230910541F0833051
:10261000910541F440E050E00E94511203C08FEF59
:102620009FEF089580E090E0089508952F923F92E3
:102630004F925F926F927F928F929F92AF92BF92D2
:10264000CF92DF92FF920F931F93CF93DF93CDB77B
:10265000DEB726970FB6F894DEBF0FBECDBF8C0154
:102660005B010E94640C6C010230110509F457C033
:10267000033011053CF401151105E9F00130110595
:1026800031F0CAC0063011050CF0C6C02CC0FC01E8
:10269000F7842F2D269526952370F3E0FF2211F461
:1026A00051E0F52E83E0F89EC0011124280F23503D
:1026B000F5012183B1C060E081E00E945A0A8EE5F5
:1026C00095E00E949212892B09F4A6C0F501918130
:1026D0008AE0989FC001112481569D4FBC0182E081
:1026E0000E94D00B99C049E050E0B501C8010E949A
:1026F0005112F601808191818F3F910509F008F414
:102700008BC0F5018181882311F486E08183F50176
:102710008181863008F080C088E081837DC0FC0123
:10272000428053804114510409F076C0F501828142
:10273000882309F469C0F601808091808114910496
:1027400009F46AC0F5012181822F63E00E946A25A5
:10275000F82EF394822F0E946A25892F9927880FDB
:10276000991F880F991FF82AF6012288338834E1CF
:10277000632E712C6C0C7D1C8501065F1F4FB3010D
:10278000C8010E941E2286E0FE01319611928A95B0
:10279000E9F7882D8F778983C401880F892F881FD7
:1027A000990B91958F778A83FFE7FF22FB82AE0119
:1027B0004F5F5F4F64E08FEF0E94951D60E081E006
:1027C0000E945A0A80E00E949B1ABC0182E00E948B
:1027D000D00BA20160E0C2010E94080DB4018FEF8E
:1027E0000E94C51BB801C3010E941E22211431049E
:1027F00059F09301F601478560817181C1010E9402
:102800004520F601828B938B90E0F501828188232D
:1028100009F491E0F501928380E090E026960FB6EE
:10282000F894DEBF0FBECDBFDF91CF911F910F9106
:10283000FF90DF90CF90BF90AF909F908F907F9050
:102840006F905F904F903F902F900895482F30E009
:10285000832F992787FD9095FC01E259FD4F249124
:10286000241729F03F5F222399F78FEF9FEF0895F8
:102870000895EF92FF920F931F93CF93DF93EB0195
:102880008230910509F486C08330910534F40097B5
:1028900009F43EC0019769F0BAC08430910509F48B
:1028A00043C0843091050CF470C0059709F456C0FC
:1028B000AEC00E94640C8C01FC0180819181892B47
:1028C00009F4A5C064E1E62EF12CE00EF11E8E01A4
:1028D000065F1F4F65960C171D07B8F4F70180813E
:1028E000882339F00E94261487FD03C0F7018081F8
:1028F00001C080E2F80181938F01F7018081882374
:1029000051F30894E11CF11CE6CFF80110827FC05E
:102910000E94921260E081E00E945A0A2A96BE014B
:1029200082E00E94E60B73C08981FB01E80FF11D74
:10293000EF012A9682850E9426148F5FE82FFF27D9
:10294000E7FDF095E259FD4F8491882319F4EEE6F6
:10295000F2E08491992787FD909515C08981FB014C
:10296000E80FF11DEF012A9682850E9426141816A1
:1029700014F08FE201C08150E82FFF27E7FDF095AA
:10298000E259FD4F8491888342C049E050E00E94A3
:1029900051123DC00E94640C8C01FC018281938124
:1029A000892BA9F59A81992349F489E08B8381E0E9
:1029B000888F99839F8B8A838E8B29C089818F5FB3
:1029C00089838F8B8B3018F11B821A821E8A8CE0D0
:1029D00098012C5E3F4FD901FE013A9601900D926D
:1029E0008A95E1F7F80182899389009731F047854C
:1029F000608171810E94452007C0A901F8016785A7
:102A0000808191810E94FA20F801828B938B80E073
:102A100090E0DF91CF911F910F91FF90EF9008957B
:102A20008F929F92BF92CF92DF92EF92FF920F937D
:102A30001F93CF93DF93CDB7DEB727970FB6F894E8
:102A4000DEBF0FBECDBF9C018B018230910509F422
:102A500055C0833091052CF40097C1F0019759F0CF
:102A6000C8C084309105D9F1843091050CF441C07F
:102A70000597C9F1BEC04BE050E060E270E0C801CC
:102A80000A960E941722F801158AB3C0FB018281C1
:102A9000882309F4AEC08181882309F4AAC0065FA7
:102AA0001F4FA801B90199270E9402219F938F937C
:102AB00081E695E09F938F93F2E0FF2EFF920E94B4
:102AC000260C60E081E00E945A0AB8018F2D0E9416
:102AD000E60B0F900F900F900F900F908AC0FB01A4
:102AE0008181992721C0FB01818199270E94EF21D3
:102AF0001DC049E050E00E9451127BC090E0FB01F4
:102B00008281882309F491E0F80192830E94640C89
:102B10007C01F801B280BB2061F0FC0182899389BD
:102B2000009711F0828902C00E94EB21F801818395
:102B300060C0EAE08E2E912C800E911EF8018181FA
:102B4000A401BE01695F7F4F99270E9402216C0199
:102B5000F7011282138210821182BC018FEF0E9452
:102B6000C51BF70180819181892B81F186E0FE01EF
:102B7000319611928A95E9F78C2D8F778983C6015A
:102B8000880F892F881F990B91958F778A838F8162
:102B90008F778B83AE014F5F5F4F64E08FEF0E94B2
:102BA000951D6B2D81E00E945A0A8B2D0E949B1A65
:102BB000BC0182E00E94D00B40E050E06B2DCA01C6
:102BC0000E94080DB6018FEF0E94C51BF70180819E
:102BD0009181892B59F0B401C70144960E941E22AD
:102BE000F80181819927F701828B938B8FEF9FEFFB
:102BF00002C080E090E027960FB6F894DEBF0FBECB
:102C0000CDBFDF91CF911F910F91FF90EF90DF909B
:102C1000CF90BF909F908F9008950F931F93CF9365
:102C2000DF93EC010E94640C8C01209719F022972D
:102C3000C9F03DC0CE010E949212892BC1F160E023
:102C400081E00E945A0AF80182899389892B11F048
:102C500081E001C082E00E949B1ABC0182E00E94D8
:102C6000D00B25C0FC01C281D381209701F5808162
:102C70009181892BE1F082899389892BC1F060E0F1
:102C800081E00E945A0A83E00E949B1ABC0182E004
:102C90000E94D00B84EF91E00E94DD08F801828948
:102CA00093890E941B20F801C28BD38B148A80E089
:102CB00090E0DF91CF911F910F9108951F93CF93D3
:102CC000DF93EB018230910509F440C08330910518
:102CD0002CF4009789F0019731F04CC086309105B3
:102CE0000CF048C02EC00E944E1BFC01848163E0A2
:102CF0000E946A2589833EC060E081E00E945A0AF2
:102D0000898113E0819F802D11240E94AD0B82E008
:102D100090E00E94DD0881B7612F0E946A258983B7
:102D200099279F938F9385E695E09F938F9382E0F9
:102D30008F930E94260C0F900F900F900F900F9082
:102D400019C04FEE5FEF0E94511214C08A81882390
:102D500059F00E944E1B398123E0329F90011124CB
:102D6000FC0124830E94F31A90E08A81882309F4ED
:102D700091E09A8380E090E0DF91CF911F910895D8
:102D8000EF92FF920F931F93CF93DF93CDB7DEB7F0
:102D900026970FB6F894DEBF0FBECDBF8C017B0126
:102DA0000E94640CDC018D919C911197892B39F064
:102DB000FD018785992783709070039731F060E05B
:102DC00081E00E945A0A85E03AC00230110509F4F8
:102DD000A3C0033011053CF40115110539F1013090
:102DE000110571F0F8C00430110509F493C00430E6
:102DF00011050CF4EAC00530110509F4E2C0EBC07E
:102E00008EEF9FEFF701818F928F20918901309192
:102E10008A01C90101978050944020F4F70124836E
:102E20003583D9C0F70104831583D5C060E081E004
:102E30000E945A0AF7018281882341F487E00E94A8
:102E40009B1ABC0182E00E94D00BC5C060E081E00B
:102E50000E945A0AF701848195819F938F9389E696
:102E600095E09F938F9312E01F930E94260C0F9082
:102E70000F900F900F900F90F7018381843059F4D9
:102E80008FE695E09F938F931F930E94260C0F90DF
:102E90000F900F9011C0F701808599279F938F9312
:102EA00083E795E09F938F931F930E94260C0F90CA
:102EB0000F900F900F900F90F701818D928D97FDDD
:102EC00003C067E775E00AC08E5F9F4F19F46FE794
:102ED00075E004C084E00E949B1ABC0182E00E945D
:102EE000D00B81E0F701808F868B83819927813019
:102EF00091056CF08330910524F00497029738F423
:102F000002C083E001C088E0F701878B64C0F7014D
:102F1000168A61C084E056C0F70182812481358120
:102F2000882389F441E0438380E094E0868397839B
:102F3000821793072CF481E090E0F7018483958356
:102F4000F701428348C030938A01209389012115FB
:102F50003105B9F1F70183818150823090F18C9174
:102F60008F7789838D919C91880F892F881F990B6A
:102F700091958F778A83848181508F778B832150BD
:102F80003040220F232F221F330B322F3770208522
:102F9000822F99278078907095958795382B3C8360
:102FA0002F772D831E82AE014F5F5F4F67E08FEF5B
:102FB0000E94951DF70113820E94690A8FEF9FEF0F
:102FC0000CC081E0F701838306C040E050E0B70108
:102FD000C8010E94511280E090E026960FB6F89446
:102FE000DEBF0FBECDBFDF91CF911F910F91FF903C
:102FF000EF900895CF92DF92EF92FF920F931F937D
:10300000CF93DF938C01C62F0E94810B0E944E1B31
:103010006C01CA3008F05CC0DD277E01EE0CFF1C9D
:10302000EE0CFF1C82E091E0E80EF91EF8018281AF
:10303000882311F080E001C082E00E94250AF60199
:103040008581992781309105A1F0823091051CF48A
:10305000892B39F029C08230910599F00397C9F086
:1030600023C034E0CC0FDD1F3A95E1F7C755DB4FA5
:1030700017C024E0CC0FDD1F2A95E1F7C75EDB4FB8
:103080000FC094E0CC0FDD1F9A95E1F7C757DC4FD6
:1030900007C084E0CC0FDD1F8A95E1F7C750DD4FF4
:1030A000BE0182E00E94D00BE701EA81FB813097EC
:1030B00021F0B80180E090E00995F8018689882325
:1030C00029F06789808D0E94630A02C00E94690A04
:1030D000DF91CF911F910F91FF90EF90DF90CF90F4
:1030E000089560E0E2E0F1E0482F552747FD509554
:1030F00020E030E0808199278417950711F4C901F9
:1031000008956F5F2F5F3F4F3496693098F38FEFCC
:103110009FEF08950895BF92CF92DF92EF92FF92B2
:103120000F931F93CF93DF93CDB7DEB76B970FB697
:10313000F894DEBF0FBECDBFB82E28E0281718F4D4
:1031400080E090E0B6C16E010894C11CD11C8BE1F7
:10315000F60111928A95E9F7A895EB2DFF27EE0F5E
:10316000FF1FEE0FFF1FEE5FFE4F0280F381E02D89
:10317000309721F0B60181E090E009956B2DC601F2
:103180000E94FA170E947104EB2CFF24EE0CFF1C26
:10319000EE0CFF1C82E091E0E80EF91E0E940A0A84
:1031A000AC018B30910509F495C08C30910534F455
:1031B00097FDE8CF0A970CF4FCC0D4C08331910589
:1031C00009F488C08431910524F4419709F46AC157
:1031D000D9CF8431910519F0459741F1D3CFF6014C
:1031E0008281882381F0F701228133812115310505
:1031F00031F0BE016F5F7F4F84E090E050C1F60177
:1032000081818F5F26C0F7019081F7E0FB1534F0D4
:10321000F7018481891711F4B3942FC0892F0E947C
:103220007118682F772767FD70953EC0F60182817F
:10323000882389F0F701228133812115310531F08E
:10324000BE016F5F7F4F85E090E029C1F60181816B
:10325000815081832AC16B2DF7019081BB2091F0B1
:103260002CEF3FEFE20EF31EF701808124E030E007
:10327000E20EF31E891731F4BA946B2D772767FDA0
:10328000709512C037E03B1564F0D7011496F70132
:103290008481891731F46F5F68301CF414968C9127
:1032A000F8CF772767FD7095B62EE62FFF27EE0F34
:1032B000FF1FEE0FFF1FEE5FFE4F0280F381E02D38
:1032C000309709F4F2C0BE016F5F7F4F81E090E05C
:1032D0000995EBC0F7019181992361F1092F11271D
:1032E0000E571E4FF801808118162CF0892F0E946E
:1032F0007118F8018083F7018181E82FFF27EE57CD
:10330000FE4F80810E948B18282F332727FD309590
:10331000F7018181E82FFF27EE57FE4FC90137FFE4
:1033200004C088279927821B930B808337FFBDC079
:10333000B1943AC0F701228133812115310551F052
:10334000BE016F5F7F4F82E090E0F90109959923FC
:103350007CF319C0F6018281882309F491E0F6011B
:103360009283A3C0F60182818823F1F0F7012281C4
:10337000338121153105A9F0BE016F5F7F4F83E0D6
:1033800090E0F9010995F6018281882309F08DC04A
:10339000F70122813381BE016F5F7F4F81E090E0B2
:1033A0007EC0F601128281C08B2D992787FD9095F2
:1033B00080C0F601838199278430910509F446C0C5
:1033C000853091054CF48230910539F183309105B7
:1033D00084F4019771F069C08830910551F089300B
:1033E00091051CF40597B1F160C0099709F445C037
:1033F0005CC0F60186819781892B21F48FEF9FE7CE
:1034000086839783F60186819781841795070CF44C
:103410004CC01482158282E08383F60184819581F9
:103420009C0163E0220F331F6A95E1F7280F391FD3
:10343000280F391F240F351F37FD37C0868197812C
:103440008217930794F1248335832FC0F6011086E9
:1034500085E08383F60190858AE0989F900111248E
:10346000240F351F2F3F310509F008F420878EEF18
:103470009FEFF601818F928F18C0F6018181E80FCE
:10348000F11D842F805D8287F70122813381211510
:10349000310559F0BE016F5F7F4F82E090E0F90186
:1034A000099503C080E00E9449046B2DCE0101966E
:1034B00067CE6B960FB6F894DEBF0FBECDBFDF911F
:1034C000CF911F910F91FF90EF90DF90CF90BF9021
:1034D0000895CF93C82F66E071E080E00E94890BC9
:1034E0006EE071E082E00E94890B80918201893058
:1034F00010F010928201C7FD04C08C2F0E948B181F
:103500000EC0809182010E948B18992787FD9095AB
:1035100097FF03C0909581959F4F8093820166EC41
:1035200071E080E00E94890B66EA71E082E00E940F
:10353000890BCF910895CF93C82F893018F08FE26F
:1035400098E02CC00E944E1BFC0185819927823097
:10355000910581F0833091051CF4019721F018C08A
:10356000039779F015C081E1C89FC00111248A56E4
:10357000984F14C081E1C89FC00111248350994F16
:103580000DC081E1C89FC00111248C59994F06C01C
:1035900081E1C89FC001112485539A4FCF910895AE
:1035A000882319F08CE398E008950E944E1BFC01DB
:1035B000858199278230910561F0833091051CF453
:1035C000019721F00CC0039739F009C08AEB95E010
:1035D000089589EA95E0089588E995E0089587E8D7
:1035E00095E008950895EF92FF921F93CF93DF9394
:1035F0008BE8E82E81E0F82EC0E0D0E01FE1CE019C
:103600000E94F321F70161917F01861719F0CE0125
:103610000E940C22A8951150219617FFF0CFDF9140
:10362000CF911F91FF90EF90089590919001943069
:1036300008F091E08FE0EBE8F1E011928A95E9F76C
:1036400088E180938F01909390010E94F31A08956E
:1036500040E250E060E070E08BE891E00E94FB21E6
:1036600080918D0190918E018F5F9F4F11F40E9488
:10367000151B80919001843010F0109290018AEF18
:103680009FEFA1E0B0E0ABBFFC0187918F3F21F03D
:10369000882311F080936F00089508958BE891E0DE
:1036A0000895809390010E94F31A08958CEF9FEF84
:1036B000A1E0B0E0ABBFFC0187919791A791B691D3
:1036C000B070BC01CD0108958FEF9FEFA1E0B0E095
:1036D000ABBFFC01879199270895FC018685992746
:1036E000969587959C012170307080FD02C0C901BC
:1036F000089580819181009711F081E090E0089514
:103700000895FC0182819381009711F081E090E09F
:1037100008950895CF92DF92EF92FF920F931F9337
:10372000CF93DF93C82E7B01EA010E94640C8C01C9
:10373000209711F1DD24A7016C2D80E00E94951DDA
:103740008AE080932D0302C00E947104C801FE012B
:103750000995882321F480912D038823A9F70E94DD
:10376000BD1C8111DD24C801FE010995882321F4C7
:10377000D39487E08D15F8F6DF91CF911F910F91CB
:10378000FF90EF90DF90CF900895CF93DF93CDB768
:10379000DEB726970FB6F894DEBF0FBECDBF61151A
:1037A0007105C9F086E0FE01319611928A95E9F71C
:1037B000862F8F778983660F672F661F770B71952A
:1037C000862F8F778A834DE65BE1BE016F5F7F4F67
:1037D00081E00E948A1B26960FB6F894DEBF0FBECA
:1037E000CDBFDF91CF910895CF93DF93CDB7DEB7F3
:1037F00026970FB6F894DEBF0FBECDBF61157105D9
:1038000039F14115510521F186E0FE013196119201
:103810008A95E9F7862F8F778983660F672F661F52
:10382000770B7195862F8F778A83842F8F778B8381
:10383000440F452F441F550B5195842F8F778C8350
:1038400041E85BE1BE016F5F7F4F82E00E948A1B0F
:1038500026960FB6F894DEBF0FBECDBFDF91CF9195
:103860000895F894FFCFFC0180E0482F57E02191A4
:10387000282780E0922F96958F5F20FF03C0292F85
:10388000252701C0292F8830A8F33327822F4F5FC7
:10389000483068F327FD8095992708950F931F936B
:1038A0008C010E94331CF8019085891719F080E083
:1038B00090E002C081E090E01F910F910895EF9297
:1038C000FF920F931F93CF93DF93CDB7DEB7299766
:1038D0000FB6F894DEBF0FBECDBF9C0180912601CC
:1038E00080687E010894E11CF11C898383E0F70164
:1038F000818387010E5F1F4F822F8F77F80181939D
:10390000220F232F221F330B3195822F8F77819324
:10391000862F8F7781938F01CA01892F99278695EA
:1039200086958F73808367FF02C0806480830F5FFA
:103930001F4FCA0123E0969587952A95E1F78F7767
:10394000F8018193842F8295807F8F7781938F01F7
:10395000C7010E94331CF8018083C7010E94B90689
:1039600029960FB6F894DEBF0FBECDBFDF91CF9181
:103970001F910F91FF90EF9008958091AB018823E4
:1039800019F480E090E008951092AB0181E090E09E
:1039900008950895EF92FF920F931F93CF93DF93B3
:1039A000CDB7DEB729970FB6F894DEBF0FBECDBFF7
:1039B0000E94561B7B018C0165C0A8958A818430CA
:1039C00009F060C0CE0101960E944E1C882309F4C4
:1039D00059C0D801C7018F779070A070B0702E8148
:1039E00033274427552782179307A407B50709F003
:1039F00049C0D801C70180789F73A070B07027E0DC
:103A0000B595A795979587952A95D1F72D81332759
:103A10004427552782179307A407B50799F5D801BE
:103A2000C7018070907CAF71B070FEE0B595A7952E
:103A300097958795FA95D1F72C81332744275527F9
:103A400082179307A407B507E9F4D801C70180706E
:103A50009070A07EB070E5E1B595A7959795879594
:103A6000EA95D1F72B8133274427552782179307EF
:103A7000A407B50739F489818F778093260181E007
:103A800090E007C0CE0101960E94C306009709F09E
:103A900094CF29960FB6F894DEBF0FBECDBFDF914D
:103AA000CF911F910F91FF90EF9008958091260183
:103AB000992708950F931F93CF93DF93CDB7DEB768
:103AC00029970FB6F894DEBF0FBECDBFFA01A895B7
:103AD00080912601806889836A838E010D5F1F4F64
:103AE00095E0309729F081918F77D8018C9302C0AF
:103AF000D8011C9291500F5F1F4F97FFF2CFCE015C
:103B000001960E94331CF8018083CE0101960E9429
:103B10008506992729960FB6F894DEBF0FBECDBF54
:103B2000DF91CF911F910F9108950F931F93CF9322
:103B3000DF93082F162FEA0102C00E947104AE0124
:103B4000612F802F0E945A1D8823B9F3DF91CF91F6
:103B50001F910F9108959F92AF92BF92CF92DF92E3
:103B6000EF92FF920F931F93CF93DF93CDB7DEB702
:103B70002F970FB6F894DEBF0FBECDBF24C2CE0183
:103B800001960E944E1C882309F41DC26E01089400
:103B9000C11CD11C0E94640C5C01F6016181862F5E
:103BA0009927AA27BB27FC013397E032F10508F0DB
:103BB000E0C1EA5BFF4FEE0FFF1F0590F491E02D8F
:103BC0000994F60182810E944904D3C1F6018281E1
:103BD000282F3327838199279695982F88279795A3
:103BE0008795282B392BD5018D919C9182179307AE
:103BF00009F0BFC10E947C0CBCC1F6018281A82FD4
:103C0000BB27838199279695982F88279795879525
:103C1000A82BB92B8581282F3327A901542F44279E
:103C2000550F550F868199278F77907073E0880F15
:103C3000991F7A95E1F7482B592B8781992780772F
:103C4000907034E0959587953A95E1F7482B592B7C
:103C5000683029F4BA01CD010E944B0D8AC1F601EA
:103C6000648126FD6068CD010E94080D82C1F601C5
:103C700084810E94620D7DC10E94760C7AC1F6019A
:103C80008281A82FBB27838199279695982F882713
:103C900097958795A82BB92B8581282F3327A901C4
:103CA000542F4427550F550F868199278F77907091
:103CB00003E0880F991F0A95E1F7482B592B87815C
:103CC00099278077907014E0959587951A95E1F77C
:103CD000482B592B648126FD6068CD010E94CC0CD5
:103CE00048C1F50182899389892B41F0A8E09A2E79
:103CF00082898F778A878289938907C09924D50121
:103D00008C918F778A878D919C91880F892F881F3E
:103D1000990B91958F778B87F501868580FF02C07F
:103D2000F0E19F2A0E94561B7B018C01862F8F7722
:103D30008C8767E016950795F794E7946A95D1F715
:103D40008E2D8F778D8757E016950795F794E7941A
:103D50005A95D1F78E2D8F778E8747E01695079568
:103D6000F794E7944A95D1F78E2D877089298F872C
:103D7000AE01465F5F4F6BE08FEF0E94951DF9C06B
:103D80000E94561B7B018C01DC01CB018F77907068
:103D9000A070B070F601248133274427552782177D
:103DA0009307A407B50709F00EC1D801C7018078B1
:103DB0009F73A070B07037E0B695A79597958795DB
:103DC0003A95D1F725813327442755278217930742
:103DD000A407B50709F0F7C0D801C7018070907C2F
:103DE000AF71B0702EE0B695A795979587952A95F7
:103DF000D1F7268133274427552782179307A40735
:103E0000B50709F0E0C080E090E0A0EEB0E0E82265
:103E1000F9220A231B2375E116950795F794E79479
:103E20007A95D1F72781822F9927AA27BB278770F8
:103E30009070A070B070E816F9060A071B0709F029
:103E4000C2C0922E9694969496948281A82FBB27F6
:103E5000838199279695982F882797958795A82BE2
:103E6000B92B109709F4AFC0092D112700FF09C025
:103E7000C5014496AC0160E070E0CD010E940221D2
:103E8000DC01109729F0BD01809126010E94C51B1D
:103E9000D5018D919C91892B09F495C001FF93C0A8
:103EA000F5018685816086878EC0F6018281282F84
:103EB0003327838199279695982F882797958795FB
:103EC000282B392B30932F0320932E0352C0F60159
:103ED0008281282F3327838199279695982F8827C9
:103EE00097958795282B392B3093320320933103F4
:103EF000848180933F0385818093330386818093FF
:103F000034038091300381601CC0F6013296A5E332
:103F1000B3E094E081918D93915097FFFBCF809116
:103F2000300382600EC0D6011296E5E3F3E093E021
:103F30008D9185839150319697FFFACF8091300310
:103F400084608093300315C081E08093AB0111C081
:103F50000E94311CF60182810E94C10D0AC0F60147
:103F60008281882321F00E944E1BFC0184810E94E3
:103F7000AD0BD6018C9199278F77907020912601F7
:103F800033278217930749F480912D03882329F062
:103F900080912D03815080932D03F501868599270B
:103FA000969587959C012170307080FD04C0A90111
:103FB00060E0C90106C0F5014481558160898081B6
:103FC00091810E945F1CCE0101960E94C306892B3D
:103FD00009F0D5CD2F960FB6F894DEBF0FBECDBF3A
:103FE000DF91CF911F910F91FF90EF90DF90CF90D5
:103FF000BF90AF909F900895CF93DF93CDB7DEB77A
:1040000026970FB6F894DEBF0FBECDBF36E0FE0197
:10401000319611923A95E9F74983AE014F5F5F4FB0
:104020000E94951D26960FB6F894DEBF0FBECDBF39
:10403000DF91CF910895CF93DF93CDB7DEB7269769
:104040000FB6F894DEBF0FBECDBF26E0FE0131965D
:1040500011922A95E9F7282F2F772983880F892F26
:10406000881F990B91958F778A83AE014F5F5F4FC1
:1040700063E18FEF0E94951D26960FB6F894DEBF80
:104080000FBECDBFDF91CF9108959F92AF92BF92A7
:10409000CF92DF92EF92FF920F931F93CF93DF9314
:1040A000CDB7DEB726970FB6F894DEBF0FBECDBFF3
:1040B000FC018B01942E6901672B11F0232B19F45D
:1040C00080E090E085C086E05E010894A11CB11CF0
:1040D000D5011D928A95E9F754E1E52E8E2F8F7751
:1040E0008983EE0FEF2FEE1FFF0BF1958E2F8F7749
:1040F0008A8320E08E2D99278631910501F1873141
:10410000910534F48431910549F04597C9F024C0F4
:104110008731910599F0489781F01EC0802F8F77E5
:104120008B83C801880F892F881F990B91958F77F2
:104130008C83892D8F778D830FC023E02D5F2D5FBA
:1041400092E0D5011296F601E20FF11D80818D9368
:1041500091502F5F97FFF7CF10922F0310922E03ED
:10416000FF2480912E0390912F03892B09F5AE0136
:104170004F5F5F4F6E2D8FEF0E94951D85E08093FE
:104180002D0306C080912D03882341F00E94710405
:1041900080912E0390912F03892BA1F3F3948091AA
:1041A0002E0390912F03892B19F489E08F15F8F6CF
:1041B00080912E0390912F03009751F0E0912E03F0
:1041C000F0912F03E39488E18E1508F087CFCF019B
:1041D00026960FB6F894DEBF0FBECDBFDF91CF910C
:1041E0001F910F91FF90EF90DF90CF90BF90AF9015
:1041F0009F9008959A01462FBC0180E090E00E94B4
:1042000045200895DF92EF92FF920F931F93CF9373
:10421000DF93CDB7DEB726970FB6F894DEBF0FBE9B
:10422000CDBF9C017B018A0101978F5F934008F00D
:1042300050C086E0FE01319611928A95E9F7822FEF
:104240008F778983220F232F221F330B3195822FE3
:104250008F778A8310923003DD248091300387307A
:1042600031F1AE014F5F5F4F60E18FEF0E94951D0E
:104270008FE080932D0306C080912D03882331F0B9
:104280000E947104809130038730B1F78091300330
:10429000873029F082B7992788960E94DD08D39449
:1042A00080913003873019F089E08D15D0F6809128
:1042B0003003873021F4809133038F3769F4E114A0
:1042C000F10411F0F70110820115110511F0F80148
:1042D000108280E090E018C0E114F10421F0809198
:1042E0003F03F70180830115110551F08BE0F801C0
:1042F000A3E3B3E00D9001928A95E1F7F8011386EC
:10430000809131039091320326960FB6F894DEBF68
:104310000FBECDBFDF91CF911F910F91FF90EF9016
:10432000DF9008950F931F93CF93DF93CDB7DEB740
:1043300026970FB6F894DEBF0FBECDBF062F26E03E
:10434000FE01319611922A95E9F7282F2F772983BC
:10435000880F892F881F990B91958F778A838FEF0C
:104360009FEF90932F0380932E0310E080912E03F4
:1043700090912F0397FF20C0AE014F5F5F4F602FDA
:104380008FEF0E94951D85E080932D0306C08091DC
:104390002D03882341F00E94710480912E03909197
:1043A0002F039923A4F31F5F80912E0390912F0375
:1043B00097FF02C01A3000F380912E0390912F03D3
:1043C00026960FB6F894DEBF0FBECDBFDF91CF911A
:1043D0001F910F91089561E10E949221089562E179
:1043E0000E9492210895E199FECF9FBB8EBBE09A77
:1043F00099278DB308954115510569F0DC01E199C4
:10440000FECF7FBB6EBBE09A6F5F7F4F0DB20D9208
:1044100041505040B1F70895E199FECF9FBB8EBB4C
:104420006DBB0FB6F894E29AE19A0FBE0895DC01D5
:1044300001C06D9341505040E0F70895FB01DC014D
:1044400001900D920020E1F708950F931F93CF93F1
:10445000DF93CDB7DEB72C970FB6F894DEBF0FBE53
:10446000CDBF8C0136E03C8389839A832FEF3FE7F1
:104470002D833E83CE0101960E947722AF81B885BD
:10448000A00FB11F1C922C960FB6F894DEBF0FBE82
:10449000CDBFDF91CF911F910F9108950F931F937F
:1044A000CF93DF93CDB7DEB72C970FB6F894DEBF6E
:1044B0000FBECDBF8C013EE03C8389839A832FEFF2
:1044C0003FE72D833E83CE0101960E947722AF8184
:1044D000B885A00FB11F1C922C960FB6F894DEBFC2
:1044E0000FBECDBFDF91CF911F910F9108952F92F5
:1044F0003F924F925F926F927F928F929F92AF9274
:10450000BF92CF92DF92EF92FF920F931F93CF93C0
:10451000DF93CDB7DEB762970FB6F894DEBF0FBE5C
:10452000CDBFAA24BB2465014C016D877E874F87D0
:10453000588B44245524FC0146825782838181FD97
:104540005BC28FEF9FEF6FC240FE44C2862D805347
:104550008A30E0F4F0E36F1641F42A89222329F42B
:10456000772019F480E091E08BC08AE09A89989FC7
:10457000902D1124892F860D80538A8B882314F463
:10458000EFE7EA8B43FC38C27A8836C243FE05C0A7
:10459000FA89FF2311F421E02A8B862D992787FDC4
:1045A00090958836910554F5853691050CF06BC0D1
:1045B0008835910509F4D3C089359105B4F48B325F
:1045C000910509F442C08C32910544F48032910582
:1045D00009F43FC0839709F442C0F2C18D329105BE
:1045E000D9F18E9709F440C0EBC18336910509F4E7
:1045F00054C08436910509F478C0E2C18037910532
:1046000009F4A5C08137910584F48C369105B1F188
:104610008D3691052CF48936910509F466C0D0C118
:104620008F36910509F490C0CBC18537910509F407
:1046300098C08637910524F483379105B9F1C0C13C
:104640008837910509F48BC0BBC180E190E0482A0E
:10465000592AE0E2F0E005C080E890E011C0E0E413
:10466000F0E04E2A5F2AC8C188E090E0482A592A23
:10467000EFEFFEEF4E225F221A8ABEC184E090E087
:10468000482A592AB9C10F2EFFE3AF2EF02D7A9494
:104690000F2EF3E66F2EF02D3AC1EF85F889CF018A
:1046A00002968F87988BA0807A9431C1EF85F88924
:1046B000CF0102968F87988BA080B18043FE0BC0FC
:1046C000EA898E2F992787FD9095BC01C5010E942C
:1046D0005F25898B07C0F50101900020E9F731972C
:1046E000EA19E98BF9897F1A12C142FE0BC0EF85E6
:1046F000F889CF0104968F87988B20813181428180
:1047000053810DC0EF85F889CF0102968F87988B72
:10471000808191819C01442737FD4095542F590198
:104720006A01552364F4E2E0F0E04E2A5F2AD09457
:10473000C094B094A094A11CB11CC11CD11C8FEBDF
:104740009FEF482259222BC098E0998B0AC0E0E4E1
:10475000F0E04E2A5F2A0F2EF8E76F2EF02DF0E1E1
:10476000F98B42FE0BC0EF85F889CF0104968F8745
:10477000988B20813181428153810BC0EF85F8896C
:10478000CF0102968F87988B808191819C0144276D
:10479000552759016A01EFECFFEF4E225F221E01FF
:1047A0000894211C311CF989EF2EFF2400271127C2
:1047B000C601B501A80197010E947625DC01CB0155
:1047C000F10180838A301CF0860D815203C0F10113
:1047D0008081805DF10181931F01C601B501A801AF
:1047E00097010E94762559016A012115310541057D
:1047F0005105F1F6CE010196A22CA81AC2018273CE
:104800009070892B09F07A9446FE0FC0872D992766
:1048100087FD9095F989F03131F40F2EFEEF7F2E50
:10482000F02D780E02C0782E7A9443FE12C08A8949
:10483000282F332727FD30958A2D99278217930734
:104840002CF0E7EFFFEF4E225F2203C0FA89FA193E
:10485000FA8B43FE03C02A89721A01C07A18C2017A
:1048600080789170892B69F4872D7A9418164CF40E
:10487000B40180E290E00E942C25872D7A941816CE
:10488000BCF341FE04C0B4018DE290E00BC044FED5
:1048900004C0B4018BE290E005C045FE05C0B40140
:1048A00080E290E00E942C2546FE0FC0B40180E318
:1048B00090E00E942C258989803139F4862D992732
:1048C00087FD9095B4010E942C2550FE0DC0872DC8
:1048D0007A9418164CF4B40180E390E00E942C25E1
:1048E000872D7A941816BCF343FE11C08A89982F3D
:1048F00091509A8B18165CF4B40180E390E00E940A
:104900002C258A89E82FE150EA8B1816ACF3842D08
:10491000807869F4872D7A9418164CF4B40180E2FB
:1049200090E00E942C25872D7A941816BCF3F3E6AC
:104930006F1641F48A2D992787FD9095B4010E9446
:104940002C252DC023E76216B1F489898150898B0B
:104950008F3F29F1F5018081992787FD9095089473
:10496000A11CB11CB4010E942C2599899150998BEE
:104970009F3F81F714C0CE0101962816390679F0C1
:104980008E010F5F1F4FF10182911F01992787FD53
:104990009095B4010E942C2520163106A1F7842D94
:1049A0008078A9F0872D7A9418168CF4B40180E2EF
:1049B00090E00E942C25872D7A941816BCF307C02E
:1049C000862D992787FD9095B4010E942C254424BB
:1049D000552412C0F5E26F1641F444245524439443
:1049E0001A8A7A882AE0298B07C0862D992787FDA5
:1049F0009095B4010E942C25F401838183FF08C0A7
:104A0000ED85FE85CF0101968D879E87649005C058
:104A1000ED85FE856190ED87FE87662009F094CDD7
:104A2000F4018681978162960FB6F894DEBF0FBEBF
:104A3000CDBFDF91CF911F910F91FF90EF90DF904D
:104A4000CF90BF90AF909F908F907F906F905F902E
:104A50004F903F902F9008950F931F93CF93DF9324
:104A60008C01EB018B81992781FF22C082FF14C04A
:104A70002E813F814C815D81241735073CF4A8814C
:104A8000B9810D93A883B9832E813F812F5F3F4F5A
:104A90002E833F83C8010EC0E885F985802F0995D4
:104AA000892B31F4EE81FF813196EE83FF83F2CFC3
:104AB0008FEF9FEFDF91CF911F910F910895FC0130
:104AC0006150704001900110D8F7809590958E0F3D
:104AD0009F1F0895991B79E004C0991F961708F04D
:104AE000961B881F7A95C9F780950895A1E21A2E22
:104AF000AA1BBB1BFD010DC0AA1FBB1FEE1FFF1F82
:104B0000A217B307E407F50720F0A21BB30BE40BD1
:104B1000F50B661F771F881F991F1A9469F7609518
:104B20007095809590959B01AC01BD01CF010895D2
:104B3000FFFF000100000000C01600005E1600002C
:104B4000BE1200000413010010150100161301002D
:084B5000391401000D16FF00ED
:00000001FF
